:020000040000FA
:100000004F2881010108273C031D022800340530D8
:10001000A0000120A00B092800343230A0000120EC
:10002000A00B0F2800346430A0000120A00B15287D
:10003000003483120515292007203F286A288312DF
:100040008516342007206A288312051205118512AF
:100050006A286430A10032304420851432304420B4
:100060008510A10B2B2808006430A1005A304420D1
:1000700085140A3044208510A10B36280800051687
:100080000000000005126A28A20000000000000025
:100090000000000000000000A20B452808008316A5
:1000A000013085009F0167308F0007308100831287
:1000B0000730990081309F0085015E2829200515B1
:1000C0000720292005110720342085160720342019
:1000D000851207209F149F186B2883161E08F43C76
:0E00E000031819201E08F53C03181F202420C9
:02400E00D43CA0
:00000001FF
